:100000000C9462000C948A000C948A000C948A0070
:100010000C948A000C948A000C948A000C948A0038
:100020000C948A000C948A000C948A000C948A0028
:100030000C948A000C948A000C948A000C948A0018
:100040000C945A010C948A000C948A000C948A0037
:100050000C948A000C948A000C948A000C948A00F8
:100060000C948A000C948A000000000024002700F1
:100070002A0000000000250028002B0000000000DE
:1000800023002600290004040404040404040202DA
:100090000202020203030303030301020408102007
:1000A0004080010204081020010204081020000012
:1000B0000008000201000003040700000000000027
:1000C0000000090511241FBECFEFD8E0DEBFCDBF71
:1000D00011E0A0E0B1E0EEE9FEE002C005900D9273
:1000E000A432B107D9F721E0A4E2B1E001C01D922A
:1000F000AF35B207E1F710E0C2E6D0E004C02197C7
:10010000FE010E944707C136D107C9F70E94A4012A
:100110000C944D070C940000833081F028F481305A
:1001200099F08230A9F008958730A9F08830C9F09D
:100130008430B1F4809180008F7D03C08091800075
:100140008F7780938000089584B58F7784BD08955C
:1001500084B58F7DFBCF8091B0008F778093B00006
:1001600008958091B0008F7DF9CFCF93DF93282F32
:1001700030E0F901E255FF4F8491F901E656FF4F57
:10018000D491F901EA57FF4FC491CC23A1F081111A
:100190000E948C00EC2FF0E0EE0FFF1FE458FF4FA1
:1001A000A591B491EC91ED2381E090E009F480E019
:1001B000DF91CF91089580E090E0FACF1F93CF9325
:1001C000DF93282F30E0F901E255FF4F8491F901C8
:1001D000E656FF4FD491F901EA57FF4FC491CC2363
:1001E000A9F0162F81110E948C00EC2FF0E0EE0F89
:1001F000FF1FEE58FF4FA591B4918FB7F894EC9183
:10020000111108C0D095DE23DC938FBFDF91CF9111
:100210001F910895DE2BF8CFCF93DF9390E0FC0180
:10022000E656FF4F24918A579F4FFC018491882303
:10023000C9F090E0880F991FFC01E859FF4FA59184
:10024000B491FC01EE58FF4FC591D49161110DC0DE
:100250009FB7F8948C91209582238C9388812823D2
:1002600028839FBFDF91CF910895623051F49FB7EB
:10027000F8943C91822F809583238C93E8812E2BD8
:10028000EFCF8FB7F894EC912E2B2C938FBFEACF42
:100290008E50806480937C0080917A00806480938B
:1002A0007A0080917A0086FDFCCF80917800909151
:1002B000790008951F920F920FB60F9211242F9379
:1002C0003F938F939F93AF93BF9380915B019091E6
:1002D0005C01A0915D01B0915E0130915A0123E073
:1002E000230F2D3758F50196A11DB11D20935A01FA
:1002F00080935B0190935C01A0935D01B0935E01DC
:100300008091560190915701A0915801B0915901E7
:100310000196A11DB11D8093560190935701A093A2
:100320005801B0935901BF91AF919F918F913F9127
:100330002F910F900FBE0F901F90189526E8230F56
:100340000296A11DB11DD2CFCF93DF93CDB7DEB7FB
:1003500029970FB6F894DEBF0FBECDBF789484B551
:10036000826084BD84B5816084BD85B5826085BDB1
:1003700085B5816085BD80916E00816080936E003F
:100380001092810080918100826080938100809131
:1003900081008160809381008091800081608093E2
:1003A00080008091B10084608093B1008091B000A2
:1003B00081608093B00080917A00846080937A009D
:1003C00080917A00826080937A0080917A008160C7
:1003D00080937A0080917A00806880937A001092EE
:1003E000C10060E089E00E940C0161E08BE00E94A6
:1003F0000C0161E083E00E940C0162E084E00E9455
:100400000C0160E081E10E940C0160E08BE00E9441
:10041000DE0060E083E00E94DE002FB7F894809158
:100420005B0190915C01A0915D01B0915E012FBFD5
:100430008093520190935301A0935401B0935501BE
:1004400020E0222E20E0322E8FB7F89400915B013D
:1004500010915C0120915D0130915E0109831A8346
:100460002B833C838FBF8091520190915301A091C7
:100470005401B0915501081B190B2A0B3B0BC90104
:10048000B8010E94230620E030E04AE754E40E94CD
:10049000B1056D837E838F83988720E030E0A901CA
:1004A0000E94AC05181644F02FE632E143E85AE307
:1004B0002D833E834F83588789819A81AB81BC818C
:1004C0008093520190935301A0935401B09355012E
:1004D00083E10E9448017C018EE00E944801092EC0
:1004E000000CAA0BBB0B0F2C000C000B110B8E0D7C
:1004F0009F1DA01FB11F70E060E0B7FD08C0BC01E8
:1005000081159440A105B10514F06FEF73E0072E3B
:10051000000C880B990B0E94250620E030EC4FE779
:1005200054E40E94B1052B013C018FE00E94480178
:10053000BC01990F880B990B0E94250620E030EC36
:100540004FE754E40E94B1054B015C0180E10E9439
:10055000480121E0823391050CF020E02093510105
:10056000BC01990F880B990B0E94250620E030EC06
:100570004FE754E40E94B1056B017C012DE033E3A9
:100580004CEC5DE3C301B2010E94AC05E0E018163B
:100590006CF52AE836E24AE95EE3C301B2010E9443
:1005A000AC05E1E0181614F528E230EA40E05FE31C
:1005B000C301B2010E94AC05E2E01816BCF42BE0C6
:1005C0003DE244E35FE3C301B2010E94AC05E3E016
:1005D000181664F42EEE39EB47E65FE3C301B2016F
:1005E0000E94AC05E4E018160CF4E5E0F0E0EE0F34
:1005F000FF1FE85EFE4F408051802DE033E34CEC5E
:100600005DE3C501B4010E94AC05E0E018166CF58D
:100610002AE836E24AE95EE3C501B4010E94AC056E
:10062000E1E0181614F528E230EA40E05FE3C50186
:10063000B4010E94AC05E2E01816BCF42BE03DE2E8
:1006400044E35FE3C501B4010E94AC05E3E0181682
:1006500064F42EEE39EB47E65FE3C501B4010E9476
:10066000AC05E4E018160CF4E5E014E0E19FF001BD
:100670001124E050FF4F80809180A280B38020E061
:1006800030E0A901C701B6010E94AC0587FD9CC1FD
:1006900020E030E040E85FE3C701B6010E94D506E4
:1006A000181634F4C12CD12C80E8E82E8FE3F82EF4
:1006B00020E030E048E453E4C701B6010E94DA06C6
:1006C00020E030E040EA52E40E9440056B017C01EA
:1006D00081E10E94B5003C01019709F06AC0809158
:1006E000350190913601892B09F063C08FB7F894DA
:1006F00040915B0150915C0160915D0170915E01E0
:100700008FBF8091310190913201A0913301B0915E
:1007100034018A019B01081B190B2A0B3B0BD901E1
:10072000C8014093310150933201609333017093BB
:1007300034012091300114E0219FF0011124EC5D7F
:10074000FE4F80839183A283B3832F5F233008F011
:100750003FC1209330010091240110912501209187
:100760002601309127016091280170912901809123
:100770002A0190912B01600F711F821F931F00911E
:100780002C0110912D0120912E0130912F01600F2D
:10079000711F821F931F23E030E040E050E00E9471
:1007A0001D0520934D0130934E0140934F0150930E
:1007B0005001709236016092350180915101882379
:1007C00009F409C160914D0170914E0180914F0172
:1007D00090915001611571058105910509F4FBC0E7
:1007E0000E94230620E030E04AE754E40E94B1056D
:1007F0006B017C0189E00E94B5008130910541F4D4
:1008000001E0098720914B0130914C01232B09F025
:10081000198690934C0180934B0184E00E94B500AF
:100820001092490110924A0190914801891771F084
:100830008093480129813A814B815C812093430157
:100840003093440140934501509346018091430108
:1008500090914401A0914501B091460109811A810E
:100860002B813C81081B190B2A0B3B0BD901C801BA
:1008700040913F01509140016091410170914201CE
:10088000481759076A077B0708F0BFC080914701E6
:1008900090914801891709F4B8C0909347018111DC
:1008A00003C021E0913009F020E02093490181301C
:1008B00009F4911180E080934A011985111102C059
:1008C0008823C9F080913701811115C021E0209360
:1008D0003701509239014092380120933E018AE05D
:1008E00097EDA3EABBE380933A0190933B01A09379
:1008F0003C01B0933D0180913701882309F452C037
:1009000000913E0109832D813E814F815885609180
:100910003A0170913B0180913C0190913D010E9410
:100920003F0560933A0170933B0180933C019093A3
:100930003D0120E030E0A9010E94AC05181694F1B9
:10094000002309F452C010923E0180913801909129
:1009500039010197909339018093380118161906CF
:100960000CF040C0A5019401C701B6010E94DA064F
:100970002AE037ED43EA5BE30E943F056B017C010F
:1009800020E030E0A9010E94AC0587FF03C0C12C24
:10099000D12C7601C0923A01D0923B01E0923C0109
:1009A000F0923D0100913E010983602F8BE00E948F
:1009B000DE00698183E00E94DE002114310409F425
:1009C00043CD0E9400003CCDC12CD12C760170CECD
:1009D00010923001C0CEA701960160E070E080E780
:1009E00092E404CF10923701DDCF11E010933E0165
:1009F0002AE037ED43EA5BE320933A0130933B0171
:100A000040933C0150933D01CDCF198511115ACF30
:100A100072CFEFE3F1E084E190E0A0E0B0E080830A
:100A20009183A283B383148215821682178281E098
:100A300080878187128613860895A1E21A2EAA1B49
:100A4000BB1BFD010DC0AA1FBB1FEE1FFF1FA2177E
:100A5000B307E407F50720F0A21BB30BE40BF50B7B
:100A6000661F771F881F991F1A9469F76095709504
:100A7000809590959B01AC01BD01CF010895505820
:100A8000BB27AA270E9457050C949B060E948D063F
:100A900038F00E94940620F039F49F3F19F426F4B0
:100AA0000C948A060EF4E095E7FB0C948406E92F7B
:100AB0000E94AC0658F3BA176207730784079507BC
:100AC00020F079F4A6F50C94CE060EF4E0950B2EEA
:100AD000BA2FA02D0B01B90190010C01CA01A00190
:100AE0001124FF27591B99F0593F50F4503E68F1EB
:100AF0001A16F040A22F232F342F4427585FF3CF2C
:100B0000469537952795A795F0405395C9F77EF4FC
:100B10001F16BA0B620B730B840BBAF09150A1F045
:100B2000FF0FBB1F661F771F881FC2F70EC0BA0FCB
:100B3000621F731F841F48F4879577956795B79553
:100B4000F7959E3F08F0B0CF9395880F08F099274E
:100B5000EE0F9795879508950E94600608F481E04E
:100B600008950E94C5050C949B060E94940658F0B7
:100B70000E948D0640F029F45F3F29F00C94840612
:100B800051110C94CF060C948A060E94AC0668F3AF
:100B90009923B1F3552391F3951B550BBB27AA2736
:100BA00062177307840738F09F5F5F4F220F331F70
:100BB000441FAA1FA9F335D00E2E3AF0E0E832D038
:100BC00091505040E695001CCAF72BD0FE2F29D03B
:100BD000660F771F881FBB1F261737074807AB070D
:100BE000B0E809F0BB0B802DBF01FF2793585F4F82
:100BF0003AF09E3F510578F00C9484060C94CF0691
:100C00005F3FE4F3983ED4F3869577956795B79563
:100C1000F7959F5FC9F7880F911D9695879597F96E
:100C20000895E1E0660F771F881FBB1F62177307E7
:100C30008407BA0720F0621B730B840BBA0BEE1FFC
:100C400088F7E0950895E89409C097FB3EF49095E5
:100C50008095709561957F4F8F4F9F4F9923A9F095
:100C6000F92F96E9BB279395F69587957795679524
:100C7000B795F111F8CFFAF4BB0F11F460FF1BC068
:100C80006F5F7F4F8F4F9F4F16C0882311F096E9FB
:100C900011C0772321F09EE8872F762F05C06623A9
:100CA00071F096E8862F70E060E02AF09A95660F62
:100CB000771F881FDAF7880F9695879597F908951B
:100CC000990F0008550FAA0BE0E8FEEF161617065D
:100CD000E807F907C0F012161306E407F50798F0C5
:100CE000621B730B840B950B39F40A2661F0232BDE
:100CF000242B252B21F408950A2609F4A140A6955A
:100D00008FEF811D811D089597F99F6780E870E03E
:100D100060E008959FEF80EC089500240A94161671
:100D2000170618060906089500240A9412161306D9
:100D3000140605060895092E0394000C11F4882367
:100D400052F0BB0F40F4BF2B11F460FF04C06F5F83
:100D50007F4F8F4F9F4F089557FD9058440F551F59
:100D600059F05F3F71F04795880F97FB991F61F02D
:100D70009F3F79F087950895121613061406551FA4
:100D8000F2CF4695F1DF08C0161617061806991F10
:100D9000F1CF86957105610508940895E894BB2705
:100DA00066277727CB0197F908950E94600608F41B
:100DB0008FEF08950E94ED060C949B060E948D060D
:100DC00038F00E94940620F0952311F00C948406CC
:100DD0000C948A0611240C94CF060E94AC0670F382
:100DE000959FC1F3950F50E0551F629FF001729FD0
:100DF000BB27F00DB11D639FAA27F00DB11DAA1FDF
:100E0000649F6627B00DA11D661F829F2227B00D2B
:100E1000A11D621F739FB00DA11D621F839FA00DB6
:100E2000611D221F749F3327A00D611D231F849F06
:100E3000600D211D822F762F6A2F11249F5750405D
:100E40009AF0F1F088234AF0EE0FFF1FBB1F661FD8
:100E5000771F881F91505040A9F79E3F510580F0A1
:100E60000C9484060C94CF065F3FE4F3983ED4F3D1
:100E7000869577956795B795F795E7959F5FC1F745
:100E8000FE2B880F911D9695879597F90895EE0F83
:0E0E9000FF1F0590F491E02D0994F894FFCF18
:100E9E000000003F4CA6AA3E0000803E68B32A3EEA
:100EAE000000003E0000803D01000300040006002B
:040EBE000800100018
:00000001FF
